:100000000C940C030C9434030C9434030C943403BC
:100010000C9434030C9434030C9434030C94340384
:100020000C9434030C9434030C9434030C94340374
:100030000C9434030C941D0A0C9434030C94340374
:100040000C9441130C9434030C94420F0C941C0F29
:100050000C9434030C9434030C9434030C94340344
:100060000C9434030C94340300000000003E5B4FFA
:100070005B3E3E6B4F6B3E1C3E7C3E1C183C7E3C08
:10008000181C577D571C1C5E7F5E1C00183C180016
:10009000FFE7C3E7FF0018241800FFE7DBE7FF30A6
:1000A000483A060E2629792926407F050507407F14
:1000B00005253F5A3CE73C5A7F3E1C1C08081C1C87
:1000C0003E7F14227F22145F5F005F5F06097F017D
:1000D0007F006689956A606060606094A2FFA29468
:1000E00008047E040810207E201008082A1C080836
:1000F0001C2A08081E101010100C1E0C1E0C303884
:100100003E3830060E3E0E06000000000000005F84
:1001100000000007000700147F147F14242A7F2AA0
:100120001223130864623649562050000807030062
:10013000001C2241000041221C002A1C7F1C2A08AE
:10014000083E080800807030000808080808000011
:1001500060600020100804023E5149453E00427F85
:10016000400072494949462141494D331814127FD4
:100170001027454545393C4A494931412111090774
:100180003649494936464949291E000014000000F5
:1001900040340000000814224114141414140041C7
:1001A00022140802015909063E415D594E7C121184
:1001B000127C7F494949363E414141227F414141BC
:1001C0003E7F494949417F090909013E4141517337
:1001D0007F0808087F00417F41002040413F017FA8
:1001E000081422417F404040407F021C027F7F0470
:1001F00008107F3E4141413E7F090909063E4151B9
:10020000215E7F09192946264949493203017F01A8
:10021000033F4040403F1F2040201F3F4038403FA9
:10022000631408146303047804036159494D4300BF
:100230007F4141410204081020004141417F0402F6
:10024000010204404040404000030708002054548D
:1002500078407F284444383844444428384444286B
:100260007F385454541800087E090218A4A49C78BE
:100270007F0804047800447D40002040403D007F1A
:100280001028440000417F40007C047804787C08FA
:100290000404783844444438FC18242418182424CE
:1002A00018FC7C08040408485454542404043F44B3
:1002B000243C4040207C1C2040201C3C4030403CE2
:1002C00044281028444C9090907C4464544C440042
:1002D00008364100000077000000413608000201A6
:1002E0000204023C2623263C1EA1A161123A404092
:1002F000207A385454555921555579412154547810
:1003000041215554784020545579400C1E527212A8
:100310003955555559395454545939555454580030
:1003200000457C410002457D420001457C40F029AA
:100330002429F0F0282528F07C54554500205454F9
:100340007C547C0A097F493249494932324848483D
:1003500032324A4848303A4141217A3A4240207884
:10036000009DA0A07D39444444393D4040403D3C7F
:1003700024FF2424487E4943662B2FFC2F2BFF09A2
:1003800029F620C0887E0903205454794100004496
:100390007D413048484A32384040227A007A0A0A81
:1003A000727D0D19317D2629292F282629292926F4
:1003B00030484D4020380808080808080808382F39
:1003C00010C8ACBA2F102834FA00007B00000814C3
:1003D0002A142222142A1408AA005500AAAA55AAEF
:1003E00055AA000000FF00101010FF00141414FFA5
:1003F000001010FF00FF1010F010F0141414FC0097
:100400001414F700FF0000FF00FF1414F404FC14A0
:100410001417101F10101F101F1414141F00101099
:1004200010F0000000001F101010101F101010100E
:10043000F010000000FF101010101010101010FF2E
:1004400010000000FF140000FF00FF00001F101745
:100450000000FC04F414141710171414F404F4002E
:1004600000FF00F714141414141414F700F71414F4
:1004700014171410101F101F141414F4141010F07B
:1004800010F000001F101F0000001F14000000FCEF
:10049000140000F010F01010FF10FF141414FF14DB
:1004A0001010101F00000000F010FFFFFFFFFFF012
:1004B000F0F0F0F0FFFFFF0000000000FFFF0F0F63
:1004C0000F0F0F38444438447C2A2A3E147E02021F
:1004D0000606027E027E0263554941633844443C6D
:1004E00004407E201E2006027E020299A5E7A599FF
:1004F0001C2A492A1C4C7201724C304A4D4D303036
:1005000048784830BC625A463D3E494949007E0120
:1005100001017E2A2A2A2A2A44445F444440514A3F
:10052000444040444A51400000FF0103E080FF0086
:100530000008086B6B083612362436060F090F06C2
:10054000000018180000001010003040FF010100EA
:100550001F01011E00191D1712003C3C3C3C00000D
:1005600000000013018032118064260104B1020BE7
:1005700014C0020800C10105C5024130C701C1EC29
:10058000011B3A8155642A040000007F2B040000FF
:10059000009F3601C8B70100F20100E08F28242235
:1005A000312B0E53A5421618121A140332E18F177D
:1005B0001B1D0E14112CA53D09272D252B3C321394
:1005C000800A2980FF00000000240027002A000084
:1005D000000000250028002B000404040404040487
:1005E00004020202020202030303030303010204E2
:1005F00008102040800102040810200102040810A5
:1006000020000000080002010000030407000000B1
:100610000000000000003A1811241FBECFEFD8E000
:10062000DEBFCDBF11E0A0E0B1E0E4EEFCE302C02C
:1006300005900D92A23BB107D9F725E0A2EBB1E0FE
:1006400001C01D92A83CB207E1F713E0CCE0D3E073
:1006500004C02197FE010E945F1CCB30D107C9F76F
:100660000E948B130C94701E0C9400004C7F38E099
:10067000439FC001112430E043E0359527954A950A
:10068000E1F7822B932B687F962B089508952F9284
:100690003F924F925F926F927F928F929F92AF9212
:1006A000BF92CF92DF92EF92FF920F931F93CF935F
:1006B000DF93CDB7DEB72D970FB6F894DEBF0FBE30
:1006C000CDBF9D838C836A30A1F4DC0154962C91BC
:1006D00054971E968D919C911F97B8E02B9F800D8B
:1006E000911D1124EC81FD819787868715861486DC
:1006F000F1C06D3009F4EEC02C813D813D872C871F
:10070000D9011C96CD90DC901D9718968D919C91E7
:100710001997C816D906BCF0EC85FD854489242FAD
:1007200030E084859585F6E04F9F800D911D112462
:10073000AC85BD851D969C938E931C9756964C91C7
:100740004111A4C0C7C0EC85FD858684978482854D
:1007500093858816990604F7F489F983AF2EB12C96
:10076000C60126E0F29F800D911D1124181619066E
:100770009CF6C50123E0880F991F2A95E1F7880DA3
:10078000991D1816190644F6AC85BD8552960D9034
:10079000BC91A02DBD83AC83EC85FD850088F189DB
:1007A000E02DFF83EE83F5E06F9FB0011124160169
:1007B0001A829B012C193D0939872887C4010896A4
:1007C0009B878A879A81953049F0E885F985E20D03
:1007D000F31DE859FF4FA491AB8301C01B82240194
:1007E0003401BB81B0FF13C0AC85BD85ED91FC9198
:1007F000B981B13031F40084F185E02D2E813F8143
:1008000019C00288F389E02DEE80FF801EC0EC81C4
:10081000FD812E813F81E217F307F1F0AC85BD85A4
:10082000ED91FC91B981B13059F40084F185E02D4E
:100830002C813D81A301B1018C859D8509950CC05A
:100840000288F389E02DEC80FD8085019501A201ED
:10085000B6018C859D850995EB81E695EB83FFEFCD
:100860006F1A7F0A4A0C5B1C2A853B8526153705C3
:1008700009F0B7CF3A813F5F3A835FEF251A350A17
:10088000CA0CDB1C363009F09DCF46CF4AEF42033D
:10089000B001439F700D1124AC85BD8518964D9114
:1008A0005C911997460F571F481759079CF483E02E
:1008B000220F331F8A95E1F71E968D919C911F9709
:1008C000280F391F1F963C932E931E971D961C923E
:1008D0001E921C9781E090E02D960FB6F894DEBF33
:1008E0000FBECDBFDF91CF911F910F91FF90EF9081
:1008F000DF90CF90BF90AF909F908F907F906F9040
:100900005F904F903F902F900895EF92FF920F933A
:100910001F93DC011A960D911C911B9718962D912F
:100920003C911997ED91FC910288F389E02D7B01B0
:1009300040E050E060E070E009951F910F91FF905A
:10094000EF9008956F927F928F929F92AF92BF9295
:10095000CF92DF92EF92FF920F931F93CF93DF938B
:100960006C015A014801EB013B01620E731EC61572
:10097000D70574F4D601ED91FC910484F585E02D42
:1009800087019401A501BE01C60109952196EFCF0B
:10099000DF91CF911F910F91FF90EF90DF90CF905B
:1009A000BF90AF909F908F907F906F900895EF923F
:1009B000FF920F931F93260F371F21503109DC013F
:1009C000ED91FC910284F385E02D78018A0109956F
:1009D0001F910F91FF90EF900895EF92FF920F9368
:1009E0001F93240F351F21503109DC01ED91FC913B
:1009F0000284F385E02D780189019B0109951F91FF
:100A00000F91FF90EF9008956F927F928F929F9237
:100A1000AF92BF92CF92DF92EF92FF920F931F930C
:100A2000CF93DF93EC014B015A0169013801E88152
:100A3000F9810684F785E02D87010995A501460D0A
:100A4000571D41505109E881F9810684F785E02D51
:100A50009601B401CE010995E881F9810484F585F8
:100A6000E02D9301A501B401CE010995C80CD91C54
:100A7000B60161507109E881F9810484F585E02DA2
:100A80009301A501CE010995DF91CF911F910F919F
:100A9000FF90EF90DF90CF90BF90AF909F908F909E
:100AA0007F906F9008952F923F924F925F926F9236
:100AB0007F928F929F92AF92BF92CF92DF92EF92EE
:100AC000FF920F931F93CF93DF9300D000D000D0FD
:100AD000CDB7DEB72C017E836D836A015901C80151
:100AE000FC82EB824801841A950A97FE03C0919418
:100AF0008194910835012D813E81621A730A77FE37
:100B000003C0719461947108681479045CF43A2DFF
:100B10002B2D5C01832F922F3D812E81DE82CD8291
:100B2000C32ED22EAD81BE81AA16BB065CF43C2D2D
:100B30002D2D6C01832F922F3D812E81BE82AD829F
:100B4000A32EB22E85012D813E81021B130B1C01A9
:100B50002C183D0837FE03C03194219431087801E8
:100B600017FF03C03FEFE31AF30AF594E794C816A2
:100B7000D9062CF08FEF9FEF9A83898304C0A1E000
:100B8000B0E0BA83A9832D813E81A216B30624F179
:100B9000D201ED91FC910084F185E02D2B813C8107
:100BA0006814790424F44D815E81B60103C0A60166
:100BB0006D817E81C2010995E218F308F7FE06C037
:100BC00029813A81C20ED31EE00EF11E8D819E81D5
:100BD00001969E838D83D7CF26960FB6F894DEBFFD
:100BE0000FBECDBFDF91CF911F910F91FF90EF907E
:100BF000DF90CF90BF90AF909F908F907F906F903D
:100C00005F904F903F902F900895089580E090E07E
:100C100008950F931F93CF93DF932091B4012F5F1B
:100C2000322F37703093B40120FF02C020E801C09A
:100C300020E031FD2064347009F02062205FFC0167
:100C4000EC01239600E011E06485662331F070E04A
:100C5000C8010E943C1C6F5F01C060E06187322FB9
:100C6000369F030E30E0311D1124311102C016826F
:100C700002C031503683662311F06150618731968E
:100C8000CE17DF0709F7DF91CF911F910F910895DC
:100C900080E991E00895539A08950F931F93CF939D
:100CA000DF93CDB7DEB762970FB6F894DEBF0FBE05
:100CB000CDBF8C01F901DC011C968C917A8369838C
:100CC0005C834B835E834D8390819D8791819E875A
:100CD00092819F87813029F4CE0101960E940906F6
:100CE00006C01C861B861A86198618861F8283E01A
:100CF000888B1A8A198AD801ED91FC910484F585B4
:100D0000E02DBE016F5F7F4FC801099562960FB657
:100D1000F894DEBF0FBECDBFDF91CF911F910F9131
:100D200008950F931F93CF93DF93CDB7DEB76297EC
:100D30000FB6F894DEBF0FBECDBF8C01F901DC0108
:100D40001C968C917A8369835C834B835E834D838D
:100D500090819D8791819E8792819F87813029F420
:100D6000CE0101960E94090606C01C861B861A86C3
:100D7000198618861F82188A1A8A198AD801ED9155
:100D8000FC910484F585E02DBE016F5F7F4FC801A3
:100D9000099562960FB6F894DEBF0FBECDBFDF9106
:100DA000CF911F910F91089580E090E00895FC018C
:100DB000858596850895CF93DF9300D000D000D02D
:100DC000CDB7DEB7AB011C821D821E82DC01ED9126
:100DD000FC910190F081E02D19821A821B829E0104
:100DE0002F5F3F4FBE016C5F7F4F099526960FB670
:100DF000F894DEBF0FBECDBFDF91CF9108954F9223
:100E00005F926F927F928F92AF92BF92CF92DF925A
:100E1000EF920F931F93CF93DF933C01EB010E945E
:100E2000BC11F30127853089621B730B6A30710591
:100E3000B0F3F894E881F9817BB178606BB1677F9A
:100E40006BB9CA848F812C2D281B822F2F83BF84DE
:100E50004A805B801D850C85DE841F5F0F5FD39405
:100E60009E813885A984EB844181D20120E0C32F83
:100E7000522F322F3181442788943111380F08F4D2
:100E80003FEF8195889410FD430F4795889411FD9D
:100E9000430F4795889412FD430F4795889413FD9F
:100EA000430F4795889414FD430F4795889415FD8B
:100EB000430F4795889416FD430F4795889417FD77
:100EC000430F47958894232F1111242F8C0D422F07
:100ED000002C7BB900C047FF6BB930812227889472
:100EE00000C000C0002C6BB93111390F00C0002CBC
:100EF0007BB900C046FF6BB908F43FEF9195889429
:100F000000C000C0002C6BB900FD230F00C0002CF6
:100F10007BB900C045FF6BB92795889401FD230F6D
:100F200000C000C0002C6BB92795889400C0002C2D
:100F30007BB900C044FF6BB902FD230F279588944D
:100F400000C000C0002C6BB903FD230F00C0002CB3
:100F50007BB900C043FF6BB92795889404FD230F2C
:100F600000C000C0002C6BB92795889400C0002CED
:100F70007BB900C042FF6BB905FD230F279588940C
:100F800000C000C0002C6BB906FD230F00C0002C70
:100F90007BB900C041FF6BB92795889407FD230FEB
:100FA00000C000C0002C6BB92795889400C0002CAD
:100FB0007BB900C040FF6BB9432F0111422F9A0D3E
:100FC00000C000C0002C6BB900C000C0002C7BB971
:100FD00000C047FF6BB932812227889400C000C04F
:100FE000002C6BB931113C0F00C0002C7BB900C044
:100FF00046FF6BB908F43FEFEB0DF11D00C000C0D8
:10100000002C6BB9D0FC230F00C0002C7BB900C0B2
:1010100045FF6BB927958894D1FC230F00C000C011
:10102000002C6BB92795889400C0002C7BB900C0B8
:1010300044FF6BB9D2FC230F2795889400C000C0F1
:10104000002C6BB9D3FC230F00C0002C7BB900C06F
:1010500043FF6BB927958894D4FC230F00C000C0D0
:10106000002C6BB92795889400C0002C7BB900C078
:1010700042FF6BB9D5FC230F2795889400C000C0B0
:10108000002C6BB9D6FC230F00C0002C7BB900C02C
:1010900041FF6BB927958894D7FC230F00C000C08F
:1010A000002C6BB92795889400C0002C7BB900C038
:1010B00040FF6BB9432FD110422FC19500C000C033
:1010C000002C6BB9CE0D00C000C07BB900C047FF3B
:1010D0006BB931812227889400C000C0002C6BB905
:1010E0003111380F00C0002C7BB900C046FF6BB92E
:1010F00008F43FEF8195889400C000C0002C6BB9C4
:1011000010FD230F00C0002C7BB900C045FF6BB958
:101110002795889411FD230F00C000C0002C6BB9E7
:101120002795889400C0002C7BB900C044FF6BB9A0
:1011300012FD230F2795889400C000C0002C6BB9C6
:1011400013FD230F00C0002C7BB900C043FF6BB917
:101150002795889414FD230F00C000C0002C6BB9A4
:101160002795889400C0002C7BB900C042FF6BB962
:1011700015FD230F2795889400C000C0002C6BB983
:1011800016FD230F00C0002C7BB900C041FF6BB9D6
:101190002795889417FD230F00C000C0002C6BB961
:1011A0002795889400C0002C7BB900C040FF6BB924
:1011B000432F1111422F8C0D00C000C0002C6BB9C1
:1011C000119709F086CE20EE31E0D2010E94581C22
:1011D000DC01CB01F4E0B695A79597958795FA9534
:1011E000D1F720E030E0B901EAE94E9E040C611D20
:1011F0005E9E600D711D1124650D711D860F971F78
:10120000A11DB11D893E43E09407A105B10508F475
:1012100034C0885E9340A109B10942E0B695A79514
:10122000979587954A95D1F747E0849F080E211D31
:10123000949F200D311D1124290F311D6091B301A0
:1012400070E0860F971F820F931F40915B045091AF
:101250005C0460915D0470915E04292F3327420F76
:10126000531F611D711D40935B0450935C04609398
:101270005D0470935E048093B30178940E94BC1166
:10128000F301708B6787DF91CF911F910F91EF90E2
:10129000DF90CF90BF90AF908F907F906F905F90D6
:1012A0004F900895CF93DF93EC0160E08D810E9411
:1012B000331144E050E080E090E0DC011EBC0DB44E
:1012C00007FEFDCF2EB5BA2FA92F982F8827822B86
:1012D0004150510999F727702C8322E1B695A795C3
:1012E000979587952A95D1F79F70BC0180E090E093
:1012F0000E946E1920E030E040E85EE30E94AB19E6
:10130000688379838A839B8361E08D810E94331196
:10131000DF91CF910895EF92FF920F931F93CF9398
:10132000DF93EC010E941B120C811D812E813F81F5
:10133000DC01CB01801B910BA20BB30B088119813F
:101340002A813B8180179107A207B307F0F10E9421
:101350001B126C837D838E839F83CE0108960E942F
:1013600052098A89FE0194E0899FE00DF11D112444
:10137000488559856A857B85438B548B658B768B35
:101380008F5F8A3010F48A8B01C01A8A8E010D5E3D
:101390001F4F7E01EBE3EE0EF11C60E070E0CB012D
:1013A000F80121913191419151918F010E94041BCB
:1013B0000E151F05A9F720E030E040E251E40E943D
:1013C000701B6E877F87888B998BDF91CF911F91E0
:1013D0000F91FF90EF900895FC01868D882339F0DE
:1013E0006EBD00000DB407FEFDCF8EB5089528E058
:1013F00030E090E8A1A1B2A186A5462F492319F0BB
:101400004C91842B03C04C91809584238C93A3A191
:10141000B4A14C9187A5842B8C93A3A1B4A14C912A
:1014200087A5809584238C9396952150310911F7D7
:10143000089508958CBD9DBD08951F920F920FB61B
:101440000F9211242F933F934F935F936F937F934A
:101450008F939F93AF93BF93EF93FF93E0E0F0E000
:101460000995FF91EF91BF91AF919F918F917F91DE
:101470006F915F914F913F912F910F900FBE0F9001
:101480001F90189586E495E00E948B098BE095E00B
:101490000E948B0980915205882321F088E591E014
:1014A0000E94E11080911705882321F082E691E0E7
:1014B0000E94E1102091190530911A0540911B05F9
:1014C00050911C0560915405709155058091560509
:1014D000909157050E94041B20E030E040E05FE35C
:1014E0000E94AB190E94E21BCB010895EF92FF927C
:1014F0000F931F93CF93DF93EC017B018C010E5F61
:101500001F4F1B821A821D821C821F821E8240E096
:1015100050E06AEA71E0C8010E94A10E19821882A7
:101520006CE671E0C8010E94E10E198618861B86E0
:101530001A868FEFE816F80671F482E390E099833B
:10154000888360E771E0C8010E94E10E1986188661
:101550001B861A8699C08BE5E816F104BCF426E9CF
:1015600030E0D7010E94581C2AE530E040E050E00E
:101570000E94691A398328836EE771E0C8010E94CE
:10158000E10E198618868AE590E07CC085EBE816A6
:10159000F10484F486E990E09983888369E871E036
:1015A000C8010E94E10E8BE590E09987888784EB63
:1015B00090E068C081EFE816F10444F5C701FF0C24
:1015C000AA0BBB0B9C01AD01245B310941095109F8
:1015D000AAE5B0E00E94881A2CE330E040E050E039
:1015E0000E94691ADA01C9018A569F4FAF4FBF4F57
:1015F000998388836EE871E0C8010E94E10E85EB53
:1016000090E09987888780EF90E03CC08FE0E816F3
:1016100081E0F80684F480EF90E0998388836EE897
:1016200071E0C8010E94E10E81EF90E09987888700
:101630008EE091E027C0C701FF0CAA0BBB0B9C01F9
:10164000AD012E50314041095109A0E1BFEF0E9488
:10165000961A22E330E040E050E00E94691ADA0175
:10166000C90180519F4FAF4FBF4F9983888366E771
:1016700071E0C8010E94E10E8FE091E099878887B0
:1016800080E491E09B878A87CE01DF91CF911F9103
:101690000F91FF90EF900895CF93DF93EC0180912D
:1016A000B201811117C081E08093B20161E08BE04B
:1016B0000E94801161E08DE00E94801160E08CE06A
:1016C0000E94801161E08AE00E94331184E58CBDA4
:1016D0008DB58EB561E08D850E94801161E08D85AC
:1016E0000E943311CE0108960E945209888599857F
:1016F000AA85BB85FE017396EB9681939193A19386
:10170000B193EC17FD07C9F7DF91CF910895CF9200
:10171000DF92EF92FF920F931F93CF93DF936C01B1
:101720007A018B01C0E0D0E0CE15DF0581F0D80151
:101730006D918D01D601ED91FC910190F081E02D2C
:10174000C6010995892B11F02196EECF7E01C701C4
:10175000DF91CF911F910F91FF90EF90DF90CF908D
:101760000895FC01538D448D252F30E0842F90E0A7
:10177000821B930B541710F0CF960895019708958C
:10178000FC01918D828D981761F0828DDF01A80F89
:10179000B11D5D968C91928D9F5F9F73928F90E0AB
:1017A00008958FEF9FEF0895FC01918D828D98171A
:1017B00031F0828DE80FF11D858D90E008958FEF57
:1017C0009FEF0895FC01918D228D892F90E0805C20
:1017D0009F4F821B91098F739927089581E694E0AA
:1017E0000E94E20B21E0892B09F420E0822F08956A
:1017F000FC01848DDF01A80FB11DA35ABF4F2C91AE
:10180000848D90E001968F739927848FA689B7897C
:101810002C93A089B1898C91837080648C93938D73
:10182000848D981306C00288F389E02D80818F7D16
:1018300080830895EF92FF920F931F93CF93DF93CE
:10184000EC0181E0888F9B8D8C8D981305C0E88911
:10185000F989808185FD26C0F62E0B8D10E00F5F83
:101860001F4F0F731127E02E8C8DE8120CC00FB69E
:1018700007FCFACFE889F989808185FFF5CFCE0191
:101880000E94F80BF1CF8B8DFE01E80FF11DE35A9A
:10189000FF4FF0829FB7F8940B8FEA89FB89808114
:1018A00080620AC09FB7F894EE89FF896083E88957
:1018B000F98980818370806480839FBF81E090E09C
:1018C000DF91CF911F910F91FF90EF900895CF93EB
:1018D000DF93EC01888D8823C9F0EA89FB89808138
:1018E00085FD05C0A889B9898C9186FD0FC00FB60A
:1018F00007FCF5CF808185FFF2CFA889B9898C914B
:1019000085FFEDCFCE010E94F80BE7CFDF91CF919D
:10191000089580E090E0892B29F00E94EE0B811160
:101920000C9400000895EF92FF920F931F93DC0137
:101930001A960D911C911B9718962D913C91199711
:10194000ED91FC910288F389E02D7B0140E050E0AD
:1019500060E070E009951F910F91FF90EF9008955E
:101960000E944C1EAF92BF92CF92DF92EF92FF92F5
:101970000F931F93CF93DF93EC01590168012885E2
:101980003985621773070CF075C08A859B854817E7
:1019900059070CF06FC0FB01EA0DFB1D2E173F0726
:1019A0001CF45901A61AB70A9A012C0D3D1D821785
:1019B00093071CF46C01C41AD50A8D8D823091F402
:1019C0009701322F2227330F330F330FC701807E49
:1019D0009770822B932BEF2CFF24E694E694E694E9
:1019E000E82AF92A0FEF040F0C0D2FEF260F2A0D0E
:1019F000CE010E94F4108E8D882321F08F8D98A146
:101A00000E941A0AEFA1F8A5908189A9892B8083E9
:101A1000EDA1FEA1908188A98095892380831C1463
:101A20001D049CF48501101611065CF46F2DCE0187
:101A30000E94EC096E2DCE010E94EC0901501109A3
:101A4000F2CF81E0C81AD108EACFEDA1FEA19081C2
:101A500088A9892B80838E8D882361F0DF91CF91B7
:101A60001F910F91FF90EF90DF90CF90BF90AF90BC
:101A70000C94190ADF91CF911F910F91FF90EF9075
:101A8000DF90CF90BF90AF900895CF92DF92EF920A
:101A9000FF920F931F93CF93DF93EC0169017801BD
:101AA00088859985681779070CF061C02A853B8580
:101AB000421753070CF05BC09B012C0D3D1D821794
:101AC00093071CF46C01C61AD70A2FEF260F2C0DB2
:101AD000042FCE010E94F4108D8D823091F4970175
:101AE000322F2227330F330F330FC701807E9770B9
:101AF000822B932BEF2CFF24E694E694E694E82ABD
:101B0000F92A8E8D882321F08F8D98A10E941A0AC0
:101B1000EFA1F8A5908189A9892B8083EDA1FEA171
:101B2000908188A9809589238083C114D10461F0B4
:101B30006F2DCE010E94EC096E2DCE010E94EC09A2
:101B400081E0C81AD108F1CFEDA1FEA1908188A94A
:101B5000892B80838E8D882351F0DF91CF911F9147
:101B60000F91FF90EF90DF90CF900C94190ADF91C6
:101B7000CF911F910F91FF90EF90DF90CF9008953C
:101B8000CF92DF92EF92FF920F931F93CF93DF9349
:101B9000EC016901780188859985681779070CF04F
:101BA00062C08A859B85481759070CF05CC09A0172
:101BB0002C0D3D1D821793071CF46C01C41AD50A25
:101BC0000FEF040F0C0D262FCE010E94F4108D8D07
:101BD000823091F49701322F2227330F330F330FC6
:101BE000C701807E9770822B932BEF2CFF24E69405
:101BF000E694E694E82AF92A0F2D8E8D882321F0A9
:101C00008F8D98A10E941A0AEFA1F8A5908189A949
:101C1000892B8083EDA1FEA1908188A980958923DD
:101C20008083C114D10461F0602FCE010E94EC09C1
:101C30006E2DCE010E94EC0981E0C81AD108F1CFC7
:101C4000EDA1FEA1908188A9892B80838E8D8823A8
:101C500051F0DF91CF911F910F91FF90EF90DF90A6
:101C6000CF900C94190ADF91CF911F910F91FF90A3
:101C7000EF90DF90CF900895EF92FF920F93CF9364
:101C8000DF93EC01790177FD56C088859985681747
:101C900079070CF050C057FD4EC08A859B854817C8
:101CA00059070CF048C001E0040F21E0260FCE01D7
:101CB0000E94F4108E8D882321F08F8D98A10E94B0
:101CC0001A0AEFA1F8A5908189A9892B8083EDA13B
:101CD000FEA1908188A98095892380838D8D823093
:101CE00091F49701322F2227330F330F330FC7019F
:101CF000807E9770822B932BEF2CFF24E694E69442
:101D0000E694E82AF92A6F2DCE010E94EC096E2D87
:101D1000CE010E94EC09EDA1FEA1908188A9892B3A
:101D200080838E8D882339F0DF91CF910F91FF90C2
:101D3000EF900C94190ADF91CF910F91FF90EF90E3
:101D40000895EF92FF920F931F93CF93DF93EC01CF
:101D50007B018A0188819981009729F02A813B8142
:101D600024173507F8F4B8016F5F7F4F0E94861D76
:101D7000009759F0998388831B830A832C813D81C6
:101D8000232B81F4FC0110820DC08881998100977A
:101D900011F00E94FD1C198218821D821C821B8278
:101DA0001A8207C01D830C83B701888199810E9424
:101DB0005A1ECE01DF91CF911F910F91FF90EF90AE
:101DC0000895CF93DF93EC016115710559F0FB0184
:101DD00001900020E9F73197AF01461B570B0E9495
:101DE000A10E0CC088819981009711F00E94FD1C02
:101DF000198218821D821C821B821A82CE01DF91F9
:101E0000CF910895FC01808191810C94FD1C611596
:101E1000710579F0FB0101900020E9F73197AF01DE
:101E2000461B570BDC01ED91FC910280F381E02D04
:101E3000099480E090E008951F920F920FB60F92E0
:101E400011242F933F934F935F936F937F938F93BF
:101E50009F93AF93BF93EF93FF9381E694E00E942B
:101E6000F80BFF91EF91BF91AF919F918F917F916F
:101E70006F915F914F913F912F910F900FBE0F90F7
:101E80001F9018951F920F920FB60F9211242F9347
:101E90008F939F93EF93FF93E0917104F0917204FD
:101EA0008081E0917704F091780482FD12C09081E6
:101EB00080917A048F5F8F7320917B04821751F099
:101EC000E0917A04F0E0EF59FB4F958F80937A040C
:101ED00001C08081FF91EF919F918F912F910F9081
:101EE0000FBE0F901F9018951F93CF93DF93EC01B7
:101EF000162F8E8D882321F08F8D98A10E941A0AAB
:101F0000EFA1F8A5908189A9892B8083EDA1FEA17D
:101F1000908188A9809589238083612FCE010E94BA
:101F2000EC09EDA1FEA1908188A9892B80838E8D7B
:101F3000882329F0DF91CF911F910C94190ADF912A
:101F4000CF911F9108951F93CF93DF93EC01162F2C
:101F50008E8D882321F08F8D98A10E941A0AEFA1FF
:101F6000F8A5908189A9809589238083EDA1FEA1A0
:101F7000908188A9809589238083612FCE010E945A
:101F8000EC09EDA1FEA1908188A9892B80838E8D1B
:101F9000882329F0DF91CF911F910C94190ADF91CA
:101FA000CF911F910895611102C060E201C061E20A
:101FB0000C94A30FEF92FF920F931F9320919A0519
:101FC0002223B9F1FA01AC0100919805109199050D
:101FD0006115710591F48E179F0724F49F01281B4A
:101FE000390B04C09C012E1B3F0BAF0160E070E079
:101FF00081E895E00E94C00D1CC08E179F0781F4F8
:102000001616170624F49B0160E070E004C0222736
:102010003327261B370B81E895E00E94450D09C048
:1020200078018F019B0160E070E081E895E00E94FB
:1020300053051F910F91FF90EF900895242F462F85
:10204000682F81E895E00E943603E1E8F5E021E0A1
:10205000218F908F878B918B808B938B828B0895B0
:1020600020919A052223D9F0109297052091980586
:102070003091990530939205209391053093940502
:102080002093930570938E0560938D055093900572
:1020900040938F05BC0181E895E00C94070F0895EB
:1020A0000F931F93CF93DF93FC01C481D5812097B9
:1020B00019F4FB01108211C0415051094C175D0702
:1020C00008F4EA018B01FC0160817181AE01C80155
:1020D0000E94611EC00FD11F1882DF91CF911F9106
:1020E0000F9108950F931F93CF93DF93CDB7DEB772
:1020F00062970FB6F894DEBF0FBECDBF8C01CB0147
:10210000F8011182108213821282158214824AE031
:10211000BE016F5F7F4F0E943919BE016F5F7F4F15
:10212000C8010E94E10E62960FB6F894DEBF0FBEA2
:10213000CDBFDF91CF911F910F9108958F929F9204
:10214000AF92BF920F931F93CF93DF93CDB7DEB7BC
:10215000A1970FB6F894DEBF0FBECDBF19A24230D3
:1021600008F44AE08E010F5D1F4F842E912CA12CA4
:10217000B12CA50194010E94D21AE62FB901CA011F
:1021800001501109EA3014F4E05D01C0E95CD801A6
:10219000EC93232B242B252B61F7B80181E694E0E7
:1021A0000E94070FA1960FB6F894DEBF0FBECDBFF9
:1021B000DF91CF911F910F91BF90AF909F908F9023
:1021C0000895CF93DF93BC0181E694E00E94070F4E
:1021D000EC0168EA71E081E694E00E94070F8C0F41
:1021E0009D1FDF91CF910895EF92FF920F931F9360
:1021F000CF93DF93EC01E62E142FF22E6AE20E94B9
:10220000A30F60E0CE010E94740F6AA96E0DCE018B
:102210000E94740F60E0CE010E94740F6AA96F0DD6
:10222000CE010E94740F6BE2CE010E94A30F60E00A
:10223000CE010E94740F6BA9610FCE010E94740F32
:1022400060E0CE010E94740F6BA9600FCE010E9466
:10225000740F6CE2CE01DF91CF911F910F91FF902F
:10226000EF900C94A30F90E0FC01EF5FF94F2491E5
:10227000FC01E351FA4F3491FC01E752FA4FE4912B
:10228000EE2309F43CC0222339F1233091F038F4D5
:102290002130A9F0223001F584B58F7D12C027309E
:1022A00091F02830A1F02430B9F4809180008F7D26
:1022B00003C0809180008F77809380000DC084B52B
:1022C0008F7784BD09C08091B0008F7703C0809163
:1022D000B0008F7D8093B000F0E0EE0FFF1FE15360
:1022E000FA4FA591B4919FB7F894611104C08C91F5
:1022F0003095382302C0EC913E2B3C939FBF08954C
:10230000CF93DF9390E0FC01E351FA4F2491FC015D
:10231000E752FA4F8491882361F190E0880F991F6A
:10232000FC01EB53FA4FC591D491FC01E153FA4FF4
:10233000A591B491611109C09FB7F8948881209547
:1023400082238883EC912E230BC0623061F49FB707
:10235000F8948881322F309583238883EC912E2B3B
:102360002C939FBF06C08FB7F894E8812E2B28834B
:102370008FBFDF91CF9108953FB7F8948091B60554
:102380009091B705A091B805B091B90526B5A89B65
:1023900005C02F3F19F00196A11DB11D3FBFBA2FF7
:1023A000A92F982F8827820F911DA11DB11DBC0157
:1023B000CD0142E0660F771F881F991F4A95D1F71C
:1023C00008958F929F92AF92BF92CF92DF92EF9239
:1023D000FF926B017C010E94BC114B015C01C11496
:1023E000D104E104F104F1F00E94BC11DC01CB0145
:1023F00088199909AA09BB09883E9340A105B1052E
:1024000070F321E0C21AD108E108F10888EE880EC5
:1024100083E0981EA11CB11CC114D104E104F10495
:1024200019F7DDCFFF90EF90DF90CF90BF90AF9086
:102430009F908F9008952FB7F89460915B047091EE
:102440005C0480915D0490915E042FBF08953F92DB
:102450004F925F926F927F928F929F92AF92BF92B4
:10246000CF92DF92EF92FF920F931F93CF93DF9360
:1024700000D01F92CDB7DEB7F82E80910105909164
:102480000205A0910305B0910405892B8A2B8B2BA3
:10249000E9F00E94BC110091C0051091C105209186
:1024A000C2053091C305DC01CB01801B910BA20B4F
:1024B000B30B0091010510910205209103053091A5
:1024C000040580179107A207B307B8F20E94BC1158
:1024D0006093C0057093C1058093C2059093C305B6
:1024E000E0910905F0910A05309759F040910505F2
:1024F0005091060560910705709108058F2D09958B
:10250000F82E00915F04109160044F2C512C612C27
:10251000712C0115110509F45FC0D8011C96EC90CF
:102520001C978091FF04909100058436910510F46A
:102530001C961C92D801ED91FC91A280B380198267
:102540001A821B82F11014C0F801458556856281FC
:1025500073819E012F5F3F4FC801F5010995D80196
:102560001C96EC921C9714960D911C911597D1CF47
:10257000F8013696CE0101966C01480199E0890E6A
:10258000911C2191222309F132803320F1F0822F16
:1025900090E0A0E0B0E09C01AD012F5F3F4F4F4FB6
:1025A0005F4FC301B2010E94181C9B01AC01832D37
:1025B00090E0A0E0B0E0BC01CD016F5F7F4F8F4F96
:1025C0009F4F0E94181CD6018C93BFEFCB1ADB0AD9
:1025D000E815F905B1F6B8CF8091BE059091BF0519
:1025E0008C010F5F1F4F1093BF050093BE054997E5
:1025F0009CF10E941B124B015C0188EE93E0089F46
:10260000B001099F700D189F700D1124072E000C4A
:10261000880B990BC090BA05D090BB05E090BC0523
:10262000F090BD05A50194012C193D094E095F09E3
:102630000E94D21A309300052093FF041092BF0528
:102640001092BE050E941B126093BA057093BB05E1
:102650008093BC059093BD050F900F900F90DF9174
:10266000CF911F910F91FF90EF90DF90CF90BF908F
:10267000AF909F908F907F906F905F904F903F9022
:1026800008951F920F920FB60F9211242F933F932C
:102690008F939F93AF93BF9380915B0490915C0461
:1026A000A0915D04B0915E043091B50523E0230F45
:1026B0002D3720F40196A11DB11D05C026E8230F7A
:1026C0000296A11DB11D2093B50580935B049093E4
:1026D0005C04A0935D04B0935E048091B605909174
:1026E000B705A091B805B091B9050196A11DB11D1E
:1026F0008093B6059093B705A093B805B093B9053C
:10270000BF91AF919F918F913F912F910F900FBEED
:102710000F901F901895CF93DF93CDB7DEB7E59755
:102720000FB6F894DEBF0FBECDBF789484B582603B
:1027300084BD84B5816084BD85B5826085BD85B565
:10274000816085BD80916E00816080936E001092E3
:10275000810080918100826080938100809181005E
:1027600081608093810080918000816080938000EF
:102770008091B10084608093B1008091B00081604D
:102780008093B00080917A00846080937A00809179
:102790007A00826080937A0080917A0081608093D1
:1027A0007A0080917A00806880937A001092C1004C
:1027B00061E084E00E94801161E085E00E94801168
:1027C00061E082E00E94801161E084E00E943311A8
:1027D00061E085E00E94331161E082E00E943311E4
:1027E000E0917104F091720482E08083E0916D04C5
:1027F000F0916E041082E0916F04F09170048FEC00
:10280000808310927904E0917504F091760486E05B
:102810008083E0917304F0917404808180618083EF
:10282000E0917304F0917404808188608083E0916A
:102830007304F0917404808180688083E091730454
:10284000F091740480818F7D808385E991E00E94FE
:10285000E1101092B4051092B30561E08091AB05D0
:102860000E94801161E08091AA050E9480118091F0
:10287000AA0590E0FC01E752FA4FE491F0E0EE0F78
:10288000FF1FE153FA4F259134913093A705209310
:10289000A605FC01E351FA4FE491E093B105809164
:1028A000AB0590E0FC01E752FA4FE491F0E0EE0F47
:1028B000FF1FE153FA4F259134913093A9052093DE
:1028C000A805FC01E351FA4FE491E093B205809131
:1028D0009F05882309F439C01FB7F8948091B5018A
:1028E000811127C0E3EEF5E08491E7EFF5E09491E4
:1028F000E82FF0E0EE0FFF1FEB53FA4FA591B491D4
:10290000EC91E92321F461E08AE00E94331161E057
:102910008AE00E9480118CB580618CBD8CB580648A
:102920008CBD61E08DE00E94801161E08BE00E942F
:1029300080118091B5018F5F8093B5011FBF80E545
:102940008093A0051092A10549C061E08091AE0579
:102950000E94801161E08091AD050E9480118091FC
:10296000AE0590E0FC01E752FA4FE491F0E0EE0F83
:10297000FF1FE153FA4FA591B491B093A505A09321
:10298000A405FC01E351FA4F84918093B005209196
:10299000AD0530E0F901E752FA4FE491F0E0EE0FB7
:1029A000FF1FE153FA4F459154915093A305409373
:1029B000A205F901E351FA4FE491E093AF059C9130
:1029C000E82FE095E923EC93E091A205F091A305AF
:1029D00090818091AF05809589238083E091A60541
:1029E000F091A70590818091B1058095892380831E
:1029F0008091AC05882321F161E00E94801161E0A3
:102A00008091AC050E94331164EF71E080E090E0AA
:102A10000E94E11160E08091AC050E94331164EFE7
:102A200071E080E090E00E94E11161E08091AC05EE
:102A30000E94331164EF71E080E090E00E94E111A8
:102A4000E3E6F5E0B49004E615E0BB2009F439C0F4
:102A5000F801649181E895E00E94A30F6801F2E01B
:102A6000CF0ED11CF80131960491202F2078A22E90
:102A70000F774601102F115050F0F401649181E856
:102A800095E00E94740FFFEF8F1A9F0AF4CFC601E2
:102A9000800F911D8C01A11002C0BA94D6CF6C0199
:102AA0009FEFC91AD90AF801649170E06F3F710570
:102AB00011F464EF71E080E090E00E94E111860182
:102AC000ECCF66E381E895E00E94A30F11E010933C
:102AD000960568EA81E895E00E94740F80EA90E02C
:102AE00090938A058093890580E890E090938C0507
:102AF00080938B0560E070E081E895E00E94930C84
:102B000086E495E00E944C0B8BE095E00E944C0B14
:102B10008091C901811144C01092BB011092BA0189
:102B20008FEF8093BE018093BF018093C00180939B
:102B3000C1018093C2018093C3011093C40110921C
:102B4000C6011092C5011092BD011092BC01809186
:102B50005F0490916004892B31F488EB91E09093AD
:102B6000600480935F04E091B601F091B701309763
:102B700021F088EB91E09583848388EB91E090933A
:102B8000B7018093B6011092C8011092C7018AE183
:102B900091E09093B9018093B80181E08093C901DD
:102BA000539A81E594E09093BB018093BA0181E050
:102BB00090E09093C6018093C501809101059091AA
:102BC0000205A0910305B0910405843CF9E09F073C
:102BD000A105B10520F484EC99E0A0E0B0E0809379
:102BE000010590930205A0930305B093040510928C
:102BF000510410925204109253048091FE040E94DA
:102C0000271281E080935A041092550410925404C4
:102C10000E941B12609356047093570480935804CB
:102C20009093590430E4432E55245394612C712C15
:102C300080915A04811101C0FFCF0E941B120091A4
:102C400056041091570420915804309159040851AA
:102C50001C4F2F4F3F4F0617170728073907A8F5B6
:102C60000E941B126093560470935704809358047B
:102C70009093590400915404109155040E94420A03
:102C8000000F111FF801EF52FE4F91838083809156
:102C900054049091550401969093550480935404E4
:102CA00062EA71E081E694E00E94070F60915404AB
:102CB0007091550480E090E04AE00E949E1068EA1E
:102CC00071E081E694E00E94070F0E94420A4C01E5
:102CD0006091540470915504CE0145960E94760A85
:102CE0000E94420A2D893E89255031098217930797
:102CF0009CF48FEF8093510410925204109253046D
:102D00008091FE040E94271260E084E00E9433114B
:102D100060E085E00E9433110E94420A2D893E89BD
:102D2000281739079CF41092510480E880935204CC
:102D3000109253048091FE040E94271261E084E007
:102D40000E94331161E085E00E943311A090540489
:102D5000B0905504C50165E070E00E94281C6C012C
:102D6000892B09F080C1E12CF12C00E810E020EA69
:102D700030E040E050E060E070E081E895E00E94E3
:102D8000B20C0D891E89B401CE0187960E94721083
:102D900043E050E0BE016D5C7F4FCE0187960E94FC
:102DA0005010B501CE0181960E94721043E050E0B0
:102DB000BE01605D7F4FCE0181960E945010B80128
:102DC000CE0101960E94721043E050E0BE01635DA7
:102DD0007F4FCE0101960E9450104FEF6FEF8FEFA3
:102DE0000E941E1082E08093950540E050E060E074
:102DF00070E0CE01C3960E94301040E050E067E3DF
:102E000070E0CE01C0960E94301040E050E06EE6C7
:102E100070E0CE018D960E9430104FEF60E080E0B0
:102E20000E941E1041E150E060EA70E081E190E014
:102E30000E94DA0F42E150E060EA70E082E190E047
:102E40000E94DA0FCE0101960E94020FCE018196F8
:102E50000E94020FCE0187960E94020F4FEF6FEF84
:102E60008FEF0E941E10812C912C54014AE0C50165
:102E7000B4010E949E1068EA71E081E694E00E942D
:102E8000070FB601CE0101960E94760A09811A81C8
:102E9000CE0103960E94020F80919A058823C9F003
:102EA000E0909805F09099059801A6EABFEF0E947E
:102EB000501CA30192010E94691ABA01A901435949
:102EC0005F4F6F4F7F4F9701B40181E895E00E94FB
:102ED0003C0E2FEF821A920AA20AB20A82E0C80EB2
:102EE000D11C92E4C91691E0D90609F0BFCFE09059
:102EF0005404F09055041AA219A21CA21BA21EA2EF
:102F00001DA26F89788D6115710531F04B8D5C8D37
:102F1000CE0181960E94A10E44E150E0BE016F5F98
:102F20007F4FCE0181960E9450104FEF6FEF8FEFD1
:102F30000E941E1081E08093950549E150E060E019
:102F400070E0CE0101960E94301040E060E08FEF0B
:102F50000E941E1001ED11E0812C912C5401C12C16
:102F6000D12CEC14FD04BCF14AE0C501B4010E946F
:102F70009E1068EA71E081E694E00E94070F80915C
:102F80009A058823E9F02090980530909905F8017A
:102F9000A081B18126EA3FEF4FEF5FEF0E94881AD0
:102FA000A30192010E94691ABA01A90143595F4F16
:102FB0006F4F7F4F9101B60181E895E00E943C0E72
:102FC000FFEFCF1ADF0A0C5F1F4F2FEF821A920A12
:102FD000A20AB20AC6CFCE0181960E94020F1AA29F
:102FE00019A21CA21BA21EA21DA246E050E06BEA81
:102FF00071E0CE0181960E94A10E44E150E0BE0135
:103000006F5F7F4FCE0181960E9450104FEF6FEFA0
:103010008FEF0E941E1082E08093950542E750E0FA
:1030200060E070E0CE0101960E9430104FEF60E04A
:1030300080E00E941E106091890570918A054EE61D
:1030400050E08EE690E00E94DA0F60918905709161
:103050008A054FE650E08FE690E00E94DA0FCE013D
:1030600081960E94020FCE0147960E94020F0E9495
:10307000890CDECD109264041092630488EE93E014
:10308000A0E0B0E08093650490936604A093670489
:10309000B09368048CE291E09093620480936104A1
:1030A00085EC90E090936E0480936D0484EC90E046
:1030B0009093700480936F0480EC90E0909372047E
:1030C0008093710481EC90E0909374048093730476
:1030D00082EC90E0909376048093750486EC90E007
:1030E000909378048093770410927A0410927B0472
:1030F00010927C0410927D048FEF8093FE04109256
:1031000000051092FF0410920A05109209058FEF36
:103110009FEFDC018093050590930605A0930705BA
:10312000B0930805109284051092830520E830E0E2
:10313000309386052093850540EA50E0509388053A
:10314000409387051092960510928E0510928D057A
:103150001092900510928F0581E0809395056FEF96
:103160007FEF70939405609393057093920560933D
:1031700091058093970590E59093A0051092A10585
:103180009AE09093AA0599E09093AB0598E090930C
:10319000AC0580939F051092AE051092AD058EE3AD
:1031A00091E0909382058093810550938A05409326
:1031B000890530938C0520938B0586E08093530519
:1031C0001092520510924E0510924F051092500524
:1031D0001092510584E690E0A0E0B0E080934605AF
:1031E00090934705A0934805B093490510924A056E
:1031F00010924B0510924C0510924D05E9E5F5E053
:1032000081E895E011921192119211928E179F0709
:10321000C9F71092580587E080931805109217059A
:1032200010921305109214051092150510921605B0
:1032300084E690E0A0E0B0E080930B0590930C054D
:10324000A0930D05B0930E0510920F051092100576
:103250001092110510921205EEE1F5E01192119213
:103260001192119285E0E634F807C1F710921D051E
:103270000895BB274A3031F4992322F4BDE290959A
:1032800081959F4F0C944519BB27FB015527AA2711
:10329000880F991FAA1FA41710F0A41B83955051E3
:1032A000B9F7A05DAA3308F0A95DA193009779F75B
:1032B000B111B1931192CB010C945E19DC01FC01A8
:1032C000672F71917723E1F7329704C07C916D935A
:1032D00070836291AE17BF07C8F30895E89409C0E0
:1032E00097FB3EF490958095709561957F4F8F4F39
:1032F0009F4F9923A9F0F92F96E9BB279395F6954F
:10330000879577956795B795F111F8CFFAF4BB0FCC
:1033100011F460FF1BC06F5F7F4F8F4F9F4F16C030
:10332000882311F096E911C0772321F09EE8872FBA
:10333000762F05C0662371F096E8862F70E060E076
:103340002AF09A95660F771F881FDAF7880F9695EF
:10335000879597F908950E94BE190C942F1A0E9420
:10336000211A38F00E94281A20F0952311F00C94AD
:10337000181A0C941E1A11240C94631A0E94401AF5
:1033800070F3959FC1F3950F50E0551F629FF001B8
:10339000729FBB27F00DB11D639FAA27F00DB11DD1
:1033A000AA1F649F6627B00DA11D661F829F22275A
:1033B000B00DA11D621F739FB00DA11D621F839FE1
:1033C000A00D611D221F749F3327A00D611D231FB7
:1033D000849F600D211D822F762F6A2F11249F5705
:1033E00050409AF0F1F088234AF0EE0FFF1FBB1F08
:1033F000661F771F881F91505040A9F79E3F5105C7
:1034000080F00C94181A0C94631A5F3FE4F3983E12
:10341000D4F3869577956795B795F795E7959F5F70
:10342000C1F7FE2B880F911D9695879597F9089502
:1034300097F99F6780E870E060E008959FEF80EC67
:10344000089500240A94161617061806090608950A
:1034500000240A9412161306140605060895092E70
:103460000394000C11F4882352F0BB0F40F4BF2BDF
:1034700011F460FF04C06F5F7F4F8F4F9F4F08951F
:1034800057FD9058440F551F59F05F3F71F0479515
:10349000880F97FB991F61F09F3F79F087950895FA
:1034A000121613061406551FF2CF4695F1DF08C019
:1034B000161617061806991FF1CF86957105610536
:1034C00008940895E894BB2766277727CB0197F9DE
:1034D0000895052E97FB1EF400940E94801A57FD54
:1034E00007D00E94D21A07FC03D04EF40C94801A25
:1034F00050954095309521953F4F4F4F5F4F089520
:1035000090958095709561957F4F8F4F9F4F08954F
:103510000E94F41AA59F900DB49F900DA49F800D5A
:10352000911D11240895B7FF0C94881A0E94881ADF
:10353000821B930B08952F923F924F925F926F924E
:103540007F928F929F92AF92BF92CF92DF92EF9233
:10355000FF920F931F93CF93DF93CDB7DEB7CA1BB4
:10356000DB0B0FB6F894DEBF0FBECDBF09942A88DF
:10357000398848885F846E847D848C849B84AA8487
:10358000B984C884DF80EE80FD800C811B81AA8114
:10359000B981CE0FD11D0FB6F894DEBF0FBECDBFDF
:1035A000ED010895A1E21A2EAA1BBB1BFD010DC05F
:1035B000AA1FBB1FEE1FFF1FA217B307E407F507E3
:1035C00020F0A21BB30BE40BF50B661F771F881FBF
:1035D000991F1A9469F760957095809590959B0155
:1035E000AC01BD01CF010895A29FB001B39FC001FE
:1035F000A39F700D811D1124911DB29F700D811D1F
:103600001124911D08955058BB27AA270E941B1B07
:103610000C942F1A0E94211A38F00E94281A20F0C8
:1036200039F49F3F19F426F40C941E1A0EF4E09519
:10363000E7FB0C94181AE92F0E94401A58F3BA17A6
:10364000620773078407950720F079F4A6F50C94B8
:10365000621A0EF4E0950B2EBA2FA02D0B01B901C2
:1036600090010C01CA01A0011124FF27591B99F0F8
:10367000593F50F4503E68F11A16F040A22F232F04
:10368000342F4427585FF3CF469537952795A79554
:10369000F0405395C9F77EF41F16BA0B620B730BFB
:1036A000840BBAF09150A1F0FF0FBB1F661F771F6C
:1036B000881FC2F70EC0BA0F621F731F841F48F421
:1036C000879577956795B795F7959E3F08F0B0CFAA
:1036D0009395880F08F09927EE0F97958795089591
:1036E0000E94841B0C942F1A0E94281A58F00E94E2
:1036F000211A40F029F45F3F29F00C94181A511157
:103700000C94631A0C941E1A0E94401A68F39923B1
:10371000B1F3552391F3951B550BBB27AA276217CD
:103720007307840738F09F5F5F4F220F331F441FDA
:10373000AA1FA9F335D00E2E3AF0E0E832D091500E
:103740005040E695001CCAF72BD0FE2F29D0660FFB
:10375000771F881FBB1F261737074807AB07B0E83E
:1037600009F0BB0B802DBF01FF2793585F4F3AF044
:103770009E3F510578F00C94181A0C94631A5F3F21
:10378000E4F3983ED4F3869577956795B795F795CA
:103790009F5FC9F7880F911D9695879597F90895B2
:1037A000E1E0660F771F881FBB1F6217730784074E
:1037B000BA0720F0621B730B840BBA0BEE1F88F75D
:1037C000E09508950E94E91B6894B1110C94631A66
:1037D00008950E94481A88F09F5798F0B92F9927AA
:1037E000B751B0F0E1F0660F771F881F991F1AF0EC
:1037F000BA95C9F714C0B13091F00E94621AB1E0D5
:1038000008950C94621A672F782F8827B85F39F0D3
:10381000B93FCCF3869577956795B395D9F73EF484
:1038200090958095709561957F4F8F4F9F4F08952C
:10383000DB018F939F930E94881ABF91AF91A29F43
:10384000800D911DA39F900DB29F900D112408959E
:10385000AA1BBB1B51E107C0AA1FBB1FA617B707B6
:1038600010F0A61BB70B881F991F5A95A9F78095D2
:103870009095BC01CD01089597FB072E16F4009496
:1038800007D077FD09D00E94281C07FC05D03EF424
:10389000909581959F4F0895709561957F4F0895FC
:1038A0000E94F41A332312F48A1B9B0B0C945A1CAB
:1038B0000E94F41AB7FF0895821B930B0895EE0F30
:1038C000FF1F0590F491E02D09940F931F93CF9360
:1038D000DF938230910510F482E090E0E091C6051C
:1038E000F091C70520E030E0A0E0B0E0309719F19A
:1038F000408151810281138148175907C8F084170C
:10390000950769F4109731F012960C93129713965D
:103910001C9327C00093C6051093C70522C021152C
:10392000310519F04217530718F49A01BD01EF0150
:10393000DF01F801DBCF21153105F9F0281B390B28
:103940002430310580F48A819B816115710521F055
:10395000FB019383828304C09093C7058093C605BF
:10396000FE01329644C0FE01E20FF31F8193919352
:1039700022503109398328833AC02091C4053091FF
:10398000C505232B41F420910201309103013093AE
:10399000C5052093C4052091000130910101211536
:1039A000310541F42DB73EB7409104015091050116
:1039B000241B350BE091C405F091C505E217F30710
:1039C000A0F42E1B3F0B2817390778F0AC014E5F8F
:1039D0005F4F2417350748F04E0F5F1F5093C50502
:1039E0004093C4058193919302C0E0E0F0E0CF01E1
:1039F000DF91CF911F910F910895CF93DF9300979F
:103A000009F481C0FC01329713821282A091C6058D
:103A1000B091C705109781F420813181820F931FE7
:103A20002091C4053091C5052817390751F5F09349
:103A3000C505E093C40567C0ED0120E030E0CE1776
:103A4000DF0740F44A815B819E0141155105F1F089
:103A5000EA01F5CFD383C28340815181840F951F42
:103A6000C817D90759F488819981840F951F029648
:103A7000918380838A819B81938382832115310581
:103A800029F4F093C705E093C6053DC0E901FB8327
:103A9000EA8349915991C40FD51FEC17FD0761F4D2
:103AA00080819181840F951F0296E9019983888313
:103AB000828193819B838A83E0E0F0E012968D916E
:103AC0009C911397009719F0FD01DC01F7CF8D91C0
:103AD0009C9111979D012E5F3F4F820F931F209164
:103AE000C4053091C5052817390769F4309729F4C2
:103AF0001092C7051092C60502C013821282B093BD
:103B0000C505A093C405DF91CF910895A0E0B0E072
:103B1000ECE8FDE10C949F1AEC01009721F4CB0135
:103B20000E94651CB4C0FC01E60FF71F9C012250E7
:103B30003109E217F30708F4A8C0D9010D911C91CF
:103B4000119706171707B0F00530110508F49BC050
:103B5000C80104978617970708F495C00250110909
:103B6000061B170B019311936D937C93CF010E9459
:103B7000FD1C89C05B01A01AB10A4C01800E911E88
:103B8000A091C605B091C705612C712CE12CF12CD8
:103B9000109709F446C08D919C911197A815B9050D
:103BA000B1F56C0142E0C40ED11CCA14DB0478F1FB
:103BB0004C018A189B08640142E0C40ED11C129685
:103BC000BC9012971396AC91B5E0CB16D10440F09F
:103BD000B282A38391828082D9016D937C9309C0C4
:103BE0000E5F1F4F800F911FF90191838083EB2D92
:103BF000FA2FE114F10431F0D7011396FC93EE9300
:103C0000129741C0F093C705E093C6053CC0681603
:103C1000790608F43C017D0112960D90BC91A02D0F
:103C2000B7CF8091C4059091C50588169906E1F437
:103C300066167706C8F48091000190910101009703
:103C400041F48DB79EB74091040150910501841B4A
:103C5000950BE817F907C8F4F093C505E093C40580
:103C6000F901718360830FC0CB010E94651C7C0148
:103C7000009759F0A801BE010E94511ECE010E947A
:103C8000FD1CC70104C0CE0102C080E090E0CDB7AA
:103C9000DEB7EEE00C94BB1A81E090E0F8940C944F
:103CA000701EFB01DC0102C001900D92415050409A
:103CB000D8F70895FB01DC0101900D920020E1F797
:103CC0000895FB01DC014150504048F001900D92F5
:103CD0000020C9F701C01D9241505040E0F70895FF
:043CE000F894FFCF86
:103CE4000000C805800000000000B00CB00CB00C4F
:103CF400DB06D706D4060000000091064D064B06ED
:103D0400DB06D7064806FF06000000001A0C870BE6
:103D1400B10B670CE20BC00BD40B0000000047038F
:103D2400870B060605063C0E5305C00D450D04051C
:103D3400B20C930CD30F36034572726F7220746306
:103D440031004572726F7220746332003430340073
:103D5400737461727420636F6F6C696E6700707244
:103D64006568656174696E6700736F616B00726585
:103D7400666C6F770048656C6C6F20576F726C646B
:103D840021007365633A20000D0A0061637469764B
:023D94006500C8
:00000001FF
